:020000040000FA
:040000008A01AE2C97
:020008008A2D3F
:10001000C92C5334503452344F344734203456347E
:1000200065347234203433342E3438340D340A3489
:10003000003450343E342034003450343E342034C4
:10004000003443345634203400343D3420340034FA
:10005000563461346C3475346534203400342134C2
:100060004F34003421344534073400344D346F3478
:100070006434653400344F344B3400344E346F34C0
:100080002034413463346B3400344F347634653477
:100090007234723475346E34073400348A01A1002E
:1000A0005720003A03190800F720210A4E28820041
:1000B0002B302C020319BF2AFE3E0319C32A5B30E2
:1000C0002C020318632D3C302C02031C632D0030DE
:1000D0008A003C302C028207612B632D612BF52CAA
:1000E000632D3D2B6C298A29632D632DC72B632D2E
:1000F000632D632D632D632D8629A92A8829F02A73
:10010000E32B632DC82B202B032C632D9329D22B9B
:10011000632D632DF02B00308A003A088207BC2D36
:10012000C42DC62DC72DCA2D9D2D9A2DAC2DA92DC0
:10013000BA2DB72DB52DB22D00308A005108820797
:100140000D2E0F2E122E1E2E212E512E542E612ECC
:10015000642E712E742E802E812E822E832E842E5C
:10016000852E862E872E882E892EA430BC00BC0BAF
:10017000B7280800BD00BD0DBD0DB520BD0BBD28C5
:100180000800561CC1280030C828561CC528FF305E
:10019000D700D801D9000330D3001430D200561054
:1001A0000800031783128D0083168C130C1483121E
:1001B0000C0803130800031783128D0075088C00C8
:1001C00083168C130C158B1355308D00AA308D00BF
:1001D0008C14000000008B17031383120D1EEE28F1
:1001E0000D12831603170C110313831208000C1E43
:1001F000F7280718FE28871AFB2800290619FE2869
:1002000099000800071286108C1E0229981C0B29E1
:10021000181218161A081A0808000D30F7200A30AC
:10022000F7200800063E831C1829313EF7200800FD
:100230002A3EF7200800A2006830F720220E0F396E
:10024000122122080F3912210800A2001E29A40041
:10025000A3012A292730A5001030A600422112212F
:100260000330A500E830A60042211221A501643028
:10027000A600422112210A30A600422112212408A0
:1002800012210800A8012608A40203184B290130F6
:10029000A302031C51292508A302031C5729A80AFD
:1002A00043292608A4070318A30A280808002608DB
:1002B000A4070318A30A2508A307280808000800B4
:1002C000A20061302202031C6A297B30220203183B
:1002D0006A29A2122208080003302D06031D832973
:1002E00083162008220424048312031D8329831605
:1002F000210623062506013A8312031D83298B015B
:1003000007308A00132F32304E200800A91608004B
:10031000A9120800E2229C210318632D01302D064A
:100320000319452AF729E2229C210318632D013085
:100330002D0603191A2ACB29831620082104031D30
:10034000A629831221304E20031408000430200215
:10035000031CB0290038031DA1292108031DA12970
:10036000831203100800C20101308316A102031C8E
:10037000A0020310A00CA10C8312C20C0310831660
:10038000A00CA10C8312C20CC20EC20CC20C8316AC
:10039000A10A831208008316220883120319D529A3
:1003A00028304E2032304E200800B3217D30831695
:1003B000A00021088312BE00C822561A08008F220E
:1003C000E622D611783042048316A00083128316E9
:1003D00023088312BE008F22E222D619F3293E3071
:1003E0004E200D2108003B304E200D2108008316C1
:1003F000220883120319FD29D02983160130A10296
:10040000031CA0028312C822561A08007C308316EF
:10041000A0048312831623088312BE007022E222F6
:10042000D619162A3E304E200D2108003B304E20B2
:100430000D21080025304E20B3217D308316A00009
:1004400021088312BE00C822561A08008F22E62215
:10045000D6110030C100703042048316A000831210
:100460004108BE008F22D619392AC10A031D302A3D
:10047000402A4108BE003E081B21E2220D2108004F
:10048000E2223E304E200D21080025304E208316FA
:100490000130A102031CA0028312C822561A0800D0
:1004A00078308316A0048312E730BE000830C10004
:1004B000C0017022D6195E2A0314602AE6220310B6
:1004C000C00DFF30BA20BE03C10B592A4008BE0040
:1004D0008316A011201583127022D6193B2A402AB8
:1004E000D6110830BF00561C732A1430D200831670
:1004F00020088312D700DA00831621088312D8005F
:10050000DA063E08D900DA060430D3005610561C2D
:10051000872AD6198E2ABF0B752A08000800D61123
:100520000830BF00561C922A1430D20083162008CF
:100530008312D700D9003E08D800D9060330D30073
:100540005610561CA12AD619A82ABF0B942A0800B7
:1005500008002D080319B52A831621088312AA0062
:10056000831620088312A90008004D30F7203D3083
:10057000F72029081B212A0825210D2108002A1609
:10058000C822D6120800861160102A12B80108008D
:100590000E30BF00DE018615601456125613D612B7
:1005A000D611C120BF0BD12A4F08DE0018305E02E1
:1005B0000318EC2A5617D6160630BF00C120BF0B11
:1005C000DE2A0800E6228611601008000A30C30007
:1005D000C120C30BE82A08008611601056160800D7
:1005E000561CF02A0E30D2002D08D3005730BB0025
:1005F000A03084000008031D632D840A0008DD007C
:10060000840A0408B4003B0884005D088000840A62
:100610000408BB0034088400AD0BFA2AAA1912237F
:10062000561008005308BF00D30A57308400DD017C
:100630000008DD06840ABF0B182B5D088000080047
:100640005330F7203D30F72044081B214508252171
:100650002030F72046081B21470825212030F720AD
:100660000608C0391B212030F72063081B216208CF
:100670002521610825210D2108002D08031D492B86
:1006800025304E203708A4003608A3002A210D216A
:100690000800831621088312B700831620088312EE
:1006A000B600003A031D5B2BB71B5B2B29120230EF
:1006B000AD06031D0800283036020318632D2916E5
:1006C000080029103C302C06031929142D08031D9D
:1006D000772B25304E20380827212F30F7207E3009
:1006E00029191C30A9180E3027210D210800831666
:1006F0002008031D862B21088312B800F030A919A9
:1007000080302919E030380503190800B801831238
:1007100032304E200800380803192910B723291851
:10072000A32B0F30A9197F3029191F303806031960
:10073000692BB80AB90B912B692B380803192914B6
:10074000BF232918912BA91DAF2B0230380603199E
:10075000B803B80BAC2B692BB90BA32B692B023058
:10076000291904303806031DA92BB801692BB901DA
:10077000B90A840A3E3000060319B82B0800B901F3
:10078000B90A840A3C3000060319C02B080008008F
:100790000230D120A9000130D120AA000330D1209D
:1007A000DF0008005F08F5000330DB202908F500B2
:1007B0000230DB202A08F5000130DB205D30F50037
:1007C0000030DB200800861160102A121F108316EB
:1007D00082309F00831281309F00D101DE0108002A
:1007E00001302D06031D0800AA129730E40083167D
:1007F000013021060319FE2B831208008312AA166A
:10080000A330E400080001302D06031D0C2C8316D4
:1008100021088312E400080064081B210D21080050
:10082000840AC0300406031403190800000860217C
:10083000800003140D3A0319080003100800112466
:10084000031808002030000603192A2C093000067E
:10085000031D0800840A1F2CAF01AE010310291BE1
:10086000812C0008423A0319902C0008483A0319D9
:100870007F2C0008443A03195D2C03189C2C30305F
:100880008002031C922C0A3000020318AC2CAF0D1E
:10089000AE0D2F08B3002E08B2000310AF0DAE0D41
:1008A0000310AF0DAE0D0310000833070318AE0A96
:1008B000AF070318AE0A3208AE0710243D2C031808
:1008C0009C2C30308002031C922C0A300002031C46
:1008D000732C11308002031CAC2C0630000203186C
:1008E000AC2C0A308007800E0430B1000310800D5C
:1008F000AF0DAE0DB10B772CB00B7F2C9C2C1024C0
:100900005F2C5F2C03189C2C30308002031C922C2F
:10091000023000020318AC2C00180314AF0DAE0D0A
:100920001024822C303080072030000603199C2CC4
:1009300009300006031DAC2C0408B400A0302D07BC
:100940002D0784002E088000840A2F088000AD0A3D
:1009500034088400031008000314080060100030FD
:100960008600EF3087008316FF308500C530860093
:10097000AF30870083128B019801831698011930DC
:1009800099002030980083129030980007308A0038
:10099000042F83168030810083128101D00106303C
:1009A000BA00D6015614C8230030D1205D3A03198D
:1009B000DF2C0C30AA00A90129156030DF00831656
:1009C00082309F00831281309F00D101DE01E1015E
:1009D000E201E3019730E400A330AA1AE4008B1689
:1009E0008B17B6010330B700B8010D2109304E2036
:1009F000AC30AB00291319302A1A1D304E200712D3
:100A00008610F401561E082D2F304E205612F82C59
:100A1000F41D1C2DF4111B303506031D132D8611FA
:100A200060102A12F82CAA1C1C2D3508F7200D3A4C
:100A3000031D1C2D0A30F72074182A2DF418262DBA
:100A4000561C022D2A1E022DAF26022D45304E20A7
:100A50000D21F82CAC3084001F240318F82C00085A
:100A600060218000AC00840AAD01AF01AE013C30D2
:100A70002C060319402D3E302C060319402D4C2D19
:100A800000083C3A031D462D9D23F82C00083E3AF1
:100A9000031D4C2D8B23F82C51302C060319672D88
:100AA0004F302C06031929171F2403185F2DB0019E
:100AB0002C240318612D06302D02031C4C2D5820C8
:100AC000F82C6325F82C32304E200D2108002A1214
:100AD00060186C2DC822D612561C672D5730BB00EB
:100AE000D3010D3000060319872D103000060319BD
:100AF000840A0008DD00D30A040AB4003B0884001D
:100B00005D088000040ABB0034088400712D1223A4
:100B10005610F82CF000030EF1000A08F200000055
:100B2000000000000408F30083010B1100006408BA
:100B300081008B289A26BA03DE2D9A260630561C91
:100B40000830BA005618DE2D5730D4000830D500D2
:100B5000DE2D9A26BA03DE2D9A260C30D20B0830F1
:100B6000BA00DE2D9A26BA03DE2DBA03DE2D9A26B0
:100B7000BA03DE2DBA01DE2D9A2654088400013016
:100B8000801F0430BA00DE2D9A26CC2DCC2D9A265B
:100B9000BA03DE2DBA03DE2DBA0154088400800D9D
:100BA000D50BDE2DD40A0830D500D30BDB2D063053
:100BB000BA005614DE2D0C30BA00DE2D8C1E0C2E21
:100BC000EA2D181218121A081A08AC30AB00F414E7
:100BD00018160C2E2B0884001A088000B500F41596
:100BE000741EF42D7412072E103A0319741608306F
:100BF0000006031D002EAC300406031DAB030C2EB3
:100C00000D300006031D072E071686147414AB0A58
:100C1000BF300406031974159C28D10A8B2ED10A03
:100C20001F158B2E1F198B2E1E08C40083161E083D
:100C30008312C50089309F00D10A8B2ED10A1F155F
:100C40008B2E1F198B2E4708CE001E08C600831658
:100C50001E088312C70091309F00D10A4E08470733
:100C6000CF00CF0C5008031D462ED61E3D2E5E0829
:100C7000053E4F020318D6158B2E561F8B2E5F088C
:100C80004F02031C8B2E6430D0008B2ED00B8B2E8A
:100C90005F084F02031C8B2E5616561386116010E8
:100CA0008B2ED10A1F158B2E1F198B2E1E08C800E4
:100CB00083161E088312C900831299309F00D10A3F
:100CC0008B2ED10A1F158B2E1F198B2E1E08CA00C2
:100CD00083161E088312CB008312A1309F00D10A15
:100CE0008B2ED10A1F158B2E1F198B2E1E08CC00A0
:100CF00083161E088312CD00831281309F00D10A13
:100D0000D10AD10AD10AD10AD10AD10AD10AD10A0B
:100D1000D10A0130D100E10F912EE20F912EE30AAA
:100D200000007308840072088A00710E8300F00EC0
:100D3000700E09000608CF39860000000000000090
:100D400000000000000000000000601C0800E01827
:100D5000AC2EE01486160800E010061608000E30CF
:100D6000D2000230D3003708D700A919D62E380890
:100D70001F39291D0F39D800291DC22E0310D80C88
:100D8000031858165817291CD816291AE22E53088A
:100D9000BF00D30A57308400DB010008DB06840A59
:100DA000BF0BCD2E5B08800056100800D30A3F30E1
:100DB000D8003808D900D9172918D9135908291A81
:100DC000E22EC72ED30A5908DA005808D90037088E
:0A0DD000D8003608C038D700C72E3F
:100E000007308A00022F000083120313061C132FE1
:100E10009927D427831203178C0883120313031D09
:100E2000132F8A0108284C30BB273E30BB270D30DA
:100E3000BB270A30BB27B0273A3A031D1B2FA3015B
:100E4000A0271F39A2000310A20CA027A000A027F2
:100E5000A1000310A00CA10CA027013A0319882FB0
:100E60002508003A031D7F2FE030200703187F2F4D
:100E7000273084002208A400A0278000840AA0272D
:100E80008000840AA40B3C2FA0272308031D962F63
:100E9000071686149927D427831203178C08831208
:100EA0000313031D592F99273F308E00FF308C000C
:100EB000C827273084002208A40007302002031C22
:100EC000672F031D7F2F0030210203187F2F20087A
:100ED000831203178F008312031321088312031751
:100EE0008D0000088C00840A00088E00840AC82740
:100EF00083120313A10F7D2FA00AA40B5D2F0716E9
:100F000086142E30BB270D30BB270A30BB271B2F82
:100F1000B027B0275330BB270D30BB270A30BB2783
:100F200099278E018C01C8278A0108284630BB27E3
:100F3000982F8312031707308F0003308D000800AD
:100F4000B027BF3E031C073E0A3EA500A50EB027F2
:100F5000BF3E031C073E0A3EA5042508A307080060
:100F600083120313071286108C1EB42F1A0807165B
:100F70008614BB270800831203130718C22F871A91
:100F8000BF2FC42F0619C22F0C1EC42F99000800B2
:100F90008316031784308C0055308D00AA308D00E5
:100FA0008C140000000008001F308F058316031703
:0C0FB00080308C000C14000000000800D1
:02400E00323F3F
:08420000000000000000600056
:00000001FF
